:020000040000FA
:060000000219FD020310CD
:030013000204FFE5
:03001B0002008D53
:03002B000202D5F9
:03005B0002050E8D
:030073000202FD89
:100080000406080C10182030406080A0C0C2AFC227
:10009000A853E6EFC28E856B8BC0D0D2D3C0E0C030
:1000A000F0C2CAA8CCA9CDD2CAD2AF758A00C3E823
:1000B000956CF8E9956DF9C3E913F9E813F8E5666D
:1000C0006007C3E913F9E813F8E97025E8956E4075
:1000D00020956E501CE582B410177C007B007A00DE
:1000E0007908900000A86AE5667004C3E813F80177
:1000F000FA900000D2A8D2AA61BAE0FDC39CC398CE
:1001000040EF98EB33FB0582E0FCC39DC39840E1D0
:1001100098EB33FB0582E0FDC39CC39840D398EB7A
:1001200033FB0582E0FCC39DC39840C598EB33FBCD
:100130000582E0FDC39CC39840B798EB33FB058272
:10014000E0FCC39DC39840A998EB33FB0582E0FD1A
:10015000C39CC398409B98EB33FB0582E0FCC39D96
:10016000C398408D98EB33FB05822175900000D237
:10017000A8D2AA61BAE0FDC39CC39840EF98EA33C5
:10018000FA0582E0FCC39DC39840E198EA33FA0582
:1001900082E0FDC39CC39840D398EA33FA0582E01D
:1001A000FCC39DC39840C598EA33FA0582E0FDC3BD
:1001B0009CC39840B798EA33FA0582E0FCC39DC31C
:1001C0009840A998EA33FA0582E0FDC39CC39840A1
:1001D0009B98EA33FA0582E0FCC39DC398408D9852
:1001E000EA33FA0582EBC46B6A54F0F9EAC454F0BE
:1001F000C3996009900000D2A8D2AA61BAEBF4C4F6
:1002000054F0F9EAF4C4540F49FAEBF4C4540FFB68
:10021000C3EAF99460FAEB9400FB5020C3E97B0039
:100220007A0079006016C3135006F9C39552600A2C
:10023000E9F552755300790080020553303A27C31F
:10024000EA94D0F8EB9407F9400BE8FAE9FB203583
:1002500009D235415A303502C235203902B235C390
:10026000EA33FAEB33FBEB2B3B3BF9C3EB13FBEA33
:1002700013FAEA29FAEB3400FB30E3047AFF7BFF40
:10028000E5255403601B202A18E55D33F9EB700760
:10029000C3E99A4002E9FAE53CC4332AFAEB340098
:1002A000FBC3EA33C4540FF8EB33C454F048F8707E
:1002B00005EA60027801C3EB13FBEA13FA90000031
:1002C000D2A8D2AAE52260021522819E900000D217
:1002D000A8D2AA61BAC0D0C0E0C2CF0541E5236070
:1002E000021523C3E554600575550041F8E5552412
:1002F00001F55550037555FFD0E0D0D032C2AF5351
:10030000E67F7592FA7593FFC22053917FD2AF3288
:10031000C0E0E58A303408856B8BF0A3D0E032D0A2
:10032000E0C2AF53E6EFC0D0C0E0C0F0D2D3D2AF4E
:100330005388EFA88AA98C758A00758C00438810B1
:1003400030331FE8C4540FFAE9C454F04AFAC31317
:100350002AFAC3E833F8E933F9E82AFAE93403FB67
:1003600061AB30320FC3E833E933FAE82AFAE934F3
:1003700000FB61AB303115E875F056A4AAF0E975C1
:10038000F056A42AFAC5F03400FB61ABE875F02BF7
:10039000A4AAF0E975F02BA42AFAC5F03400C3131F
:1003A000FBEA13FAC3EB13FBEA13FAC3EB9409500D
:1003B00009C3EA949AEB940350160522E5227002D1
:1003C0001522C3E5229432500281F275540081F562
:1003D000E522600215223036067C007D0461EAAC1D
:1003E00031AD32303A04AC33AD34C3EA9CFAEB9D04
:1003F000FB9208AE60AF61303A425007203509D217
:10040000358108303502C235303504AE62AF632025
:100410003902B235C3EA33FAEB33FBA208500AEAD9
:10042000F42401FAEBF43400FBC3EA9428FAEB94C9
:1004300000FB501478007A007B008148A208500825
:1004400078007A007B00819EE52554036019202AFC
:1004500016E55DF9EB7007C3E99A4002E9FAE53C5D
:10046000C42AFAEB3400FBEA8EF0A4F9AAF0EB8E72
:10047000F0A42AFAC5F03400FBC3EB13FDEA13F82D
:100480000FEF146004C3E833F8C3E933EA33FAEB3F
:1004900033FBDFEDEB30E20678FF7AFF7B03885415
:1004A000D230E86003755500C3E55BFC955C400203
:1004B000AC5CC3EC95545008EC75F004A4FAABF0B6
:1004C000EAF4F8EBF45403F9C3E89414FAE994005D
:1004D000FB50047A007B00885689578A588B5975DF
:1004E000230AD0F0D0E0D0D053F7DF43F74043E603
:1004F000103275230AD0F0D0E0D0D043E61032C2DB
:10050000AAD28EC2CA85CC6C85CD6DD2CA32C2AF9A
:10051000C0D0C0E0D2D3A8F9E55A30E10AE5FA200C
:10052000E13520E032A12FE5FA30E12B20E028C3AD
:10053000E55713F8E55613F5E988EAC3E55913F8CA
:10054000E55813F5FB88FC85575A53F7BFD2A830FE
:100550003402D2AA53E6EF53F7DFD0E0D0D0D2AFC7
:10056000327901801479038010790A800C791E8019
:10057000087964800479C880007817E4D5E0FDD854
:10058000FAD9F62278FF20282879A1E76023E548E8
:10059000601F74FF8548F084853FF030290375F0B3
:1005A00005A4F8C5F0600278FFC3E8955D5002A885
:1005B0005D885C22C3E54794E4E5489400E55C501F
:1005C0000314A1C5046002F55C2275E89022055E63
:1005D000C3E55E9408405330EDF4A8BDA9BE755E36
:1005E00000E9FA79A0E76041EA7006E55F601880EB
:1005F0000CC3E8955F600EE55F5005600A14800744
:100600000460FA8002E55FF55FC39569401B755B86
:10061000C0C394044013755B80C39404400B755BA6
:1006200040C394044003755B0022E55B2410500234
:1006300074FFF55B22743279A687F0A4C5F0A2F7A7
:1006400033F55D227547007548F022C2AFC2CAA8D3
:10065000CCA9CDAA4130CF010AD2CAD2AFAB42ACAD
:100660004388428943C3E89BF8E99C202808F93075
:100670002C02E15BC1B4AD448A44F9EA9DFA6006FC
:1006800078FF79FFC199AE45AF468B458C46A842AD
:10069000A943C3E89EF8E99FF9C3E54813FBE54782
:1006A00013FAE82AF547E93BF54850067547FF7508
:1006B00048FFE101AA47AB48AC47AD487E047F0242
:1006C000C3EB9404400D1E1FC3EB94084005202982
:1006D000021E1FC3ED13FDEC13FCDEF7C3EA9CFA08
:1006E000EB9DFBEF6009C3E913F9E813F8DFF7EAC4
:1006F00028FAEB39FB8A478B4850067BFF8B478BE8
:1007000048C3EB94025002D22C3028047F03E12C22
:100710007892E6FFC3E53D948240110FC3E53D9416
:10072000A040010FC3EF940640027F057E02E5481A
:10073000C4540FF9E548C454F0F8E547C4540F28F1
:10074000F8C3E89EFAE99400FB4009C3EA9401EB80
:10075000940050047A01E4FB0207A7AA47AB48EBD8
:10076000C4FEEAC4540F4EFCC3EA9CFAEB9400FBAF
:10077000C3E813C313F8EA28FAEB3400FB8A478B6B
:1007800048C3EB94024002C22C7802EBC4FE7B000B
:10079000EAC4540F4EFAC3EA98FA4005C3940150D4
:1007A000027A017892E6FF302002E1A7854E928519
:1007B0004F93D22043E680C3E49AF8E49BF9302CAF
:1007C00003020835E8FAE9FBD3E913FDE813FC88D6
:1007D0004E894FC3EF94036038EF20E00CE82CF80B
:1007E000E93DF9ECFAEDFB8013E828F8E939F9C3A3
:1007F000E82401F8E93400F97AFF7BFFC3EF9403A2
:10080000400F8A508B51884A894B8C4C8D4D020881
:100810006A885089518A4A8B4B8C4C8D4D302812F6
:100820007550F07551FF754CF0754DFF754EF075B4
:100830004FFF02086AE8FAD3E813FC884EC3EF942E
:10084000036021EF20E007E82CF8ECFA0155E828D6
:100850002401F87AFFC3EF940340098A50884A8C38
:100860004C02086A88508A4A8C4C302002016A7512
:100870003A02D22043E680E52554036034A847A914
:1008800048C3E913F9E813F8C3E913F9E813F8309A
:100890002804E92440F9C2AF53E67F759100C3E410
:1008A00098F594E499F595759104D22043E680D2A9
:1008B000AF22D221754900752000302B03752040EE
:1008C00001D0D221754900752040302B03752000DE
:1008D00078017901202C20E52554036002C221799A
:1008E00014E548C313700104F8C39414400278144B
:1008F000302804781B791B202010E549600C302833
:1009000003D53A04D222217711720549E59B544060
:10091000B52002216130280908C3E8994001180177
:10092000F720210A08C3E899400201D001F7C2214B
:1009300053E67F759100302C117594007595F8750C
:100940009104D22043E6800208D0E5487EFFC333FD
:100950004005C3334001FEC3E49E759400F5952124
:100960003FC3E5399401500201D030210201D0D8B3
:1009700002217501F7C222C2AF53E67F759100854F
:100980005094855195759104854A92854B93D22058
:1009900043E680D2AFE525540360072029020539DC
:1009A000801030220D202B0A20210715811581028D
:1009B00013B52278003021027801E53D75F007A4D7
:1009C000F9E5F028F5F0E9A2F013A2F113A2F21371
:1009D000F53DC394785003753D78C3E53D953E40A1
:1009E0000653F28F75D5FF30200221E7854C9285A2
:1009F0004D93D22043E68022203817C2AF53F2DF56
:100A0000C29643F24075D5EF43F210D2AF759F53B3
:100A1000611CC2AF53F2DFC29443F21075D5BF43DD
:100A2000F240D2AF759F53611C203817C2AF53F20A
:100A3000EF75D5DF43F220C29643F240D2AF759FE7
:100A400063611CC2AF53F2BF75D5DF43F220C2947D
:100A500043F210D2AF759F23611C203817C2AF53E9
:100A6000F2BFC29443F21075D5DF43F220D2AF75C6
:100A70009F23611CC2AF53F2EFC29643F24075D57B
:100A8000DF43F220D2AF759F63611C203817C2AFDD
:100A900053F2DF75D5BF43F240C29443F210D2AF98
:100AA000759F538077C2AF53F2DF75D5EF43F210D5
:100AB000C29643F240D2AF759F538060203817C270
:100AC000AF53F2EFC29543F22075D5BF43F240D247
:100AD000AF759F638046C2AF53F2BFC29543F22009
:100AE00075D5EF43F210D2AF759F23802F203817B2
:100AF000C2AF53F2BF75D5EF43F210C29543F22057
:100B0000D2AF759F238015C2AF53F2EF75D5BF43A7
:100B1000F240C29543F220D2AF759F63227A147BD4
:100B20007880127A107B8C800C7A0D7BB480067AE8
:100B30000B7BC88000E564D5E001227902E453F222
:100B4000DFD5E0FDD29543F220D5E0FD53F2DFD5AD
:100B5000E0FDC29543F220D5E0FDE920E005D29604
:100B600043F24030E005D29443F210E564D5E0FD55
:100B7000E920E00353F2BF30E00353F2EF7496D55F
:100B8000E0FDD9B9EAF8D5E0FDD8FBDBA853F2DFE8
:100B90002253F28F53F28F75D5FF22788076FF08AB
:100BA00076FF0876FF0876FF0876FF0876FF08765E
:100BB000090876FF087601788C76010876FF0876BA
:100BC000FF0876FF0876FF0876FF0876030876FFB1
:100BD0000876FF0876FF0876250876D0087628087C
:100BE00076500876040876FF0876020876FF0876C5
:100BF0007A0876FF0876070876010876FF0876FF00
:100C000008760008760022FA75F00CA4ABF0EAC36F
:100C100033F8740133F9E8C333F8E933F9E8C32B47
:100C2000F8E93400F9227888E6C39403D23A5002F6
:100C3000C23AC238E630E102D238A2389239788618
:100C4000E6149000809378A6F67886E6F53FC39484
:100C5000025003753F02789CE6753EFFB4020375AF
:100C60003EA0B40303753E8278A0E6F860067428BF
:100C70002409D8FCF5697896E6910788318932789D
:100C80009EE69107883389347897E69107883589FD
:100C9000367191223036117A007B007CFF7D007E18
:100CA0000091FA8B618A6022303A227896E6FA7BCC
:100CB00000789EE6FC7D00C3EA33FAEB33FBC3EC1D
:100CC00033FCED33FD7E0A91FA8B638A62789630AD
:100CD0003A02789EE6FA7B007897E6FC7D007E007B
:100CE000303A10C3EA33FAEB33FBC3EC33FCED3399
:100CF000FD7E0A91FA8B618A6022C3EC9EFCED9422
:100D000000FDC3EC9AFCED9BFDC3EC9423ED940035
:100D100050047C237D00C3EC94FFED940140047CDF
:100D2000FF7D017BFF0B7A000AEA7009C3EC33FCFC
:100D3000ED33FDA125EC8AF0A4AEF0ED8AF0A42EEF
:100D4000947C40E4EAF460DD22D236919412056D81
:100D500012056D7A007B007C10120565E5542AFAB5
:100D600074003BFBDCF37C04C3EB13FBEA13FADCFB
:100D7000F7FFEB60027FFFC23691942278A5E6F977
:100D800054037000E9540C7000E954307000E954C9
:100D9000C07000227567007568007597DE7597ADA5
:100DA0007581C043FF8075EF0675A900719175804C
:100DB000FF75F19375A4007580FF75D4FF759000E1
:100DC00075F28F75A57075900075D5FF75A60175C4
:100DD000E34075E2027191E4F8F6D8FD719B1213BD
:100DE000F378988664753001C2AF120575711D12D3
:100DF000056D712312056D712912056DB17CC2AFAD
:100E000075670075680078FA79FA308707D9FBD8DA
:100E1000F7021C009126919478988664719175E48C
:100E200007758811758E0475890975C80475910454
:100E300075D84075D90875F781759E03759601754B
:100E4000DB4275DA4275A82175E69075B801759B8D
:100E500080759D0075D10C75BC5975BB1075E88007
:100E600075B201120561D2AF753C00C23012057532
:100E7000C231C232C233C23475520075530075227A
:100E800000120571C3E522940A5002E155D2317572
:100E90002200120571C3E522940A5002E155C231C5
:100EA000D232752200120571C3E522940A5002E184
:100EB0005575E4F7758851758E017589AA758C0092
:100EC000758D00C2A9D2ABD2AA756BC0756A1475B4
:100ED0006E50C232D23475220A120571756A10C37F
:100EE000E522940A7552007553004069758E0C75A1
:100EF0006B80756A28756E2875220A120571756AED
:100F000020C3E522940A7552007553004047758E40
:100F10000C756BC0756A14756E1475220A12057112
:100F2000756A10C3E522940A755200755300402576
:100F300075E407758811758E04758909D2A9C2AB4D
:100F4000C2AAC234D233752200120571C3E52294BD
:100F50000A4002A1FE120565203003020DFEC2AF59
:100F6000711D711D711DD2AF120575203403303A09
:100F700003021014120565788CE6C3940150030235
:100F80001014E530C3940150030210147567A57561
:100F900068F17F02D2369194120571C2AFC23691C8
:100FA00094C3E554947FD2AF406A120561C2AF7119
:100FB0002FD2AFDFDFB149C3EF7897F61205751274
:100FC00014E07F0AD2369194120571C2AFC23691F5
:100FD00094C3E554947FD2AF50E8120561C2AF715B
:100FE0001D120569711DD2AFDFDAB149EF24037814
:100FF00096F6F87997E7C394234003985006E824BF
:10100000237897F6120575913AB10F120571120CFB
:1010100094020DFE756700756800120571C3E554F2
:1010200094014003020F6BC2AF120B2F120B2F1251
:101030000B2FD2AF120575753000E4F537F5380582
:1010400037E537F4703F0538789AE678191460125E
:10105000783214600D787D14600878FA1460037596
:101060003800C3E53898401D120B91120561153800
:1010700075370078998664C2AF120B2FD2AF78987B
:101080008664120571120569E5237003020DFEC323
:10109000E5549401500AC3E5529401501602103FE2
:1010A000120571E5237003020DFE755200755300A1
:1010B000021255C3E55294017017C2AF120B91781A
:1010C000998664120B1D78988664D2AF120571411F
:1010D00047C3E55294027017C2AF120B91789986FC
:1010E00064120B2378988664D2AF1205714147C30E
:1010F000E55294037017C2AF120B9178998664126F
:101100000B2978988664D2AF1205714147C3E55226
:1011100094047017C2AF120B9178998664120B2F4A
:1011200078988664D2AF1205714147C3E5529405A1
:101130007017C2AF120B9178998664120B2F7898B2
:101140008664D2AF1205714147C3E5529407701906
:10115000C3E55394065002018F7401303A027403C0
:101160007888F6C238C2394147C3E55294087019ED
:10117000C3E55394065002018F7402303A0274049E
:101180007888F6D238D2394147C3E55294097017AE
:10119000C3E55394065002018F303A0BC37888E6BA
:1011A0009402F6C23A4147C3E552940A7016C3E569
:1011B0005394065002018F203A0A7888E62402F6FA
:1011C000D23A4147C3E55294147025C3E5539406BF
:1011D0005002018FC2AF901A0B740093D2AF78887F
:1011E000F613C238C2394002D2384002D239805791
:1011F000C3E55294157038C3E5539406404FC2AF0F
:10120000901A0B740093D2AFF8B801027402B802BE
:10121000027401B803027404B8040274037888F6F7
:1012200013C238C2394002D2384002D2398018C3C2
:10123000E552940C70117567A57568F1C3E5539478
:1012400006400A913AD2AF75520075530075670097
:10125000756800018FC2AF120B91E4D2AFE4F55E66
:10126000F524F525F53D755E081205611205CA30B5
:10127000EDFDA8BDA9BEE97001F8885F1205CE7525
:101280005E08C2AF120635855D5B855D5CD2AF300E
:101290003A07C238303502D238D228753900120ADE
:1012A000BC120AED12064412064B12064412064BFB
:1012B0001206441208C21209B31209F812064B12A0
:1012C00008B2202C03120584302C031205B4120935
:1012D000B3120A2912064B1208C21209B3120A5A93
:1012E00012064B1208B21209B3120A8B12064B12E5
:1012F00008C21209B3120ABC12064B1205CA120820
:10130000B21209B3120AED1205CE12064B3028278D
:10131000855D5B79187A0CC3E53999400EC228D2F5
:10132000298A3B855D5B855D5C800CC3E554940137
:1013300040030212B361BD30291F202B1CE53B1472
:101340007006C229D22A41B3F53B203A07C3E554BF
:10135000940140030212B38064753C00203A0F7878
:10136000FA79A4E760027803C3E55598504FE52366
:10137000604B303A17203805203507800F30350292
:10138000800A202B07D22B855D5B41E378F0302B60
:1013900005855D5B7820C3E5489850030212B330A1
:1013A0002B1BC22BC238303502D238D229753B12E2
:1013B000855D5B41B3053CE554600261C0753C004E
:1013C000C2AF120B91752400752500D2AF120571C2
:1013D000120B9178A4E6600FC29643F240C2954387
:1013E000F220C29443F210C3E53C94044003020D82
:1013F000FE013A901A0D78209173E520B4550AA3A6
:101400009173E520B4AA0280137567A57568F1127F
:101410000B9B913A756700756800801D901A0378E0
:10142000807B0A9173A308DBFA901A0F788C7B1AE1
:101430009173A308DBFA901A2922C2AF91B6919357
:10144000901A0074109178A374079178A374219175
:1014500078901A0378807B0A9177A308DBFA901AB8
:101460000F788C7B1A9177A308DBFA91C991A7902A
:101470001A2922E493F622E6438F01538FFDFFC31E
:10148000E583941C400122EF8567B78568B7F05368
:101490008FFE22438F02438F018567B78568B7901F
:1014A0001A0DF0538FFC22901A0D74559178901AF2
:1014B0000E74AA9178227A3079D07820901A4091CF
:1014C00073E520F709A3DAF7227A3079D0901A4031
:1014D000E7917809A3DAF9227C05120575DCFB2275
:1014E000C2AF120B1D120B23120B29120B2F120568
:1014F00069120B1D120B23120B29120B2F120569F7
:10150000120B1D120B23120B29120B2FD2AF22C26A
:10151000AF120B2F120B29120B23120B1D12056990
:10152000120B2F120B29120B23120B1D120569121D
:0E1530000B2F120B29120B23120B1DD2AF2210
:1019FD00020D94100721FFFFFFFFFFFF09FF01FFFD
:101A0D0055AA01FFFFFFFFFF03FFFFFF25D0285061
:0D1A1D0004FF02FF7AFF0701FFFF0000FF3A
:101A400023575F4C5F32302320202020202020208D
:101A500023424C48454C492445464D3842313023B9
:101A60002020202020202020202020202020202076
:101C0000C2AFC2D37597DE7597AD7581C075A90057
:101C100043FF80752438752503B1DB7529A5752A26
:101C2000F143F18053A47FD28775D4FF75E3407DE3
:101C3000FA780379E67C10752200752300901DE880
:101C40007B06752498752501308702814820870816
:101C5000D8FBD9F9DCF781BA308708D8FBD9F9DC91
:101C6000F781BAB19BE493A3C39A6004DDC381BA40
:101C7000DBDBB18D600281317B08E493FAA3B16EA6
:101C8000DBF87A30B16E752200752300B18DEAFC65
:101C9000EBFDC3ED94FE400EB18D8A278B28ED300D
:101CA000E0048A828B83B18D7AC270D8C3ED94FE32
:101CB000601950CEBD0029EC600F7520007521FF22
:101CC000752900752A000200008100A827A92808AC
:101CD00009D804D90281DDB191EAF281D10D81A642
:101CE000C3ED94035051EDA2E092007AC5C3E582A2
:101CF0009400E583941C508C200010438F02438F86
:101D0000018529B7852AB7F0300027A827A9280818
:101D100009438F01538FFDD804D902A132C3E58353
:101D2000941C4003A3A117E28529B7852AB7F0A325
:101D3000A117538FFC81827AC1BD030CE493A3FAEF
:101D4000B152DCF8B14A81828184AA22AB23B16E00
:101D5000EBFAEA6222752608C3E52313F523E52290
:101D600013F52250066323A0632201D526EAB1DBD6
:101D7000B1DB75260AEAF4200102D287300102C2E3
:101D800087B1DBC3134002C201D526EB22B191EA31
:101D9000FB208702A191308702A196752608AE2408
:101DA000AF25C3EF13FFEE13FEB1DFB1DBC3EA13C0
:101DB0003087024480FA30E703632201C3E523132E
:101DC000F523E52213F52250066323A0632201D5F3
:101DD00026D9E52265236523F52222AE24AF250E00
:101DE0000FDEFEDFFCD20122424C48656C693437BD
:061DF0003164E8B10601B8
:00000001FF
